:10075400120100020000004005160280010001029F
:1007640000010A0600020000004001000902200006
:10077400010100A0320904000002FF000000070587
:10078400020200020007058602000200090220009E
:10079400010100A0320904000002FF000000070567
:1007A400010240000007058102400000040309041F
:1007B4002603410043004300450053002000490044
:1007C4002F004F002000500072006F00640075007D
:1007D40063007400730016035500530042002D009B
:0E07E400440049004F002D0034003800000092
:03004300020800B0
:03005300020800A0
:10080000020CA900020D4500020D2F00020D000090
:10081000020AED00020B2400020032000200420036
:1008200002005200020D9B00020D9C00020D9D0073
:10083000020D9E00020D9F00020DA000020DA100FE
:10084000020DA20002004200020DA300020DA4004E
:10085000020DA500020DA600020DA700020DA800C2
:10086000020DA90002004200020042000200420004
:10087000020DAA00020DAB00020DAC00020DAD008E
:10088000020DAE00020DAF00020DB000020DB1006E
:10089000020DB200020DB300020DB400020DB5004E
:1008A000020DB600020DB700020DB800020DB9002E
:0808B000020DBA00020DBB00AD
:0A00360000010202030304040505A3
:1008B800E4F50BF50AF509F508C203C200C202C245
:1008C80001120D18752307752454752B07752C66AE
:1008D800752107752270752907752A90752D07757A
:1008E8002EB0D2E843D82090E668E04409F090E6BC
:1008F8005CE0443DF0D2AFD20412000390E680E001
:1009080054F7F0538EF8C20330010512035EC2019A
:100918003003291200405024C203120C8420001610
:1009280090E682E030E704E020E1EF90E682E030F4
:10093800E604E020E0E4120C2C1207FE1209D58030
:01094800C7E7
:10035E0090E6B9E0700302040F14700302048C24BB
:10036E00FE700302050F24FB7003020409147003D0
:10037E000204031460731460762405600302056E94
:10038E00120D93400302057A90E6BBE024FE602234
:10039E0014603324FD601114602224067048E52396
:1003AE0090E6B3F0E5248037E52B90E6B3F0E52C2C
:1003BE00802DE52590E6B3F0E5268023E52790E62F
:1003CE00B3F0E528801990E6BAE0FF120C58AA06A1
:1003DE00A9077B01EA494B600DEE90E6B3F0EF9072
:1003EE00E6B4F002057A020573120D6D02057A125B
:1003FE000D7F02057A1207F202057A120D5B0205D5
:10040E007A120D95400302057A90E6B8E0247F60DB
:10041E001514601924027063A200E43325E0FFA2D4
:10042E0002E4334F8041E490E740F0803F90E6BC19
:10043E00E0547EFF7E00E0D394807C0040047D017A
:10044E0080027D00EC4EFEED4F2436F58274003EA8
:10045E00F583E493FF3395E0FEEF24A1FFEE34E63F
:10046E008F82F583E0540190E740F0E4A3F090E62C
:10047E008AF090E68B7402F002057A020573120D73
:10048E0097400302057A90E6B8E024FE6016240237
:10049E00600302057A90E6BAE0B40105C2000205D7
:1004AE007A02057390E6BAE0705590E6BCE0547E91
:1004BE00FF7E00E0D394807C0040047D0180027DAD
:1004CE0000EC4EFEED4F2436F58274003EF583E4CB
:1004DE0093FF3395E0FEEF24A1FFEE34E68F82F515
:1004EE0083E054FEF090E6BCE05480131313541FC7
:1004FE00FFE0540F2F90E683F0E04420F0806D80F3
:10050E0064120D99506690E6B8E024FE601924023C
:10051E00705A90E6BAE0B40104D200804F90E6BA69
:10052E00E064026047803E90E6BCE0547EFF7E00B1
:10053E00E0D394807C0040047D0180027D00EC4E6F
:10054E00FEED4F2436F58274003EF583E493FF33BF
:10055E0095E0FEEF24A1FFEE34E68F82F58380084E
:10056E00120056500790E6A0E04401F090E6A0E09D
:03057E004480F0C6
:010581002257
:0300330002004E7A
:04004E0053D8EF3262
:04004600022F000085
:0407FA0043B12022C5
:040D8F0053B1DF225B
:100D1800D200120D877580FF7590FF75B2FF75B30D
:070D28001F75B620020D8FBC
:1009D500E5336035E530452F7006752F2F7530FFEF
:1009E500E53015307002152FE530452F7004F533CD
:1009F500800FAE2FAF307C0B7DFF1206D9EF20E0C4
:100A050005120D8F80031207FAE5B190E68020E705
:0A0A150005E04408F022E054F7F079
:010A1F0022B4
:02004000D322C9
:0207FE00D32204
:020D9300D32269
:0807F20090E6BAE0F534D322D1
:100D5B0090E740E534F0E490E68AF090E68B04F0FF
:020D6B00D32291
:080D7F0090E6BAE0F531D32241
:100D6D0090E740E531F0E490E68AF090E68B04F0F0
:020D7D00D3227F
:020D9500D32267
:020D9700D32265
:020D9900D32263
:1000560075330190E678E05410C4540F4450F532DD
:1000660013E433F53590E6B9E012072E009110003F
:10007600D011010012016E30016E3101D8A201D8F3
:10008600A301D2A901A8AC0000035A90E6BEE090F5
:10009600E68BF090E6A0E020E1F9E4F512F51374A2
:1000A600402513F582E434E7F583E0FFE42513F5F4
:1000B6008274803512F583EFF00513E5137002059F
:1000C600126406451270D802035CE4F512F513E4D7
:1000D6002513F58274803512F583E0FF74402513ED
:1000E600F582E434E7F583EFF00513E513700205B6
:1000F600126406451270D802019890E6BEE090E6BA
:100106008BF090E6A0E020E1F990E6BDE0FF90E6F6
:10011600BCE04F701490E6BAE05401C454F0F59078
:1001260090E746E0F4F580800F90E746E0F4FFA301
:10013600E04FF580E0F4F590E4F512F513744025F0
:1001460013F582E434E7F583E0FFE42513F58274C2
:10015600803512F583EFF00513E51370020512647E
:1001660006451270D802035C90E740E580F0A3E5EF
:1001760090F0A3E5A0F0A3E5B0F0E5B130E4047F8C
:100186000180027F0090E6BAEFF0E5B1540F90E7E8
:1001960044F0E490E68AF090E6BEE090E68BF0024A
:1001A600035C90E6B5E054FEF090E6BFE090E68A88
:1001B600F090E6BEE090E68BF090E6BBE090E6B30A
:1001C600F090E6BAE090E6B4F002035C75350143C0
:1001D600320190E6BAE0750C00F50DA3E0FEEE42A2
:1001E6000C90E6BEE0750E00F50FA3E0FEEE420EA3
:1001F60090E6B8E064C060030202C4E50F450E70E5
:100206000302035C90E6A0E020E1F9C3E50F944009
:10021600E50E94005008850E10850F1180067510A6
:100226000075114090E6B9E0B4A335E4F512F51374
:10023600C3E5139511E5129510505EE50D2513F5EE
:1002460082E50C3512F583E0FF74402513F582E450
:1002560034E7F583EFF00513E51370D4051280D06B
:10026600E4F512F513C3E5139511E5129510501830
:1002760074402513F582E434E7F58374CDF0051355
:10028600E51370E1051280DDAD117AE779407F4014
:10029600AB07AF0DAE0C120A20E490E68AF090E6AA
:1002A6008BE511F0250DF50DE510350CF50CC3E5C4
:1002B6000F9511F50FE50E9510F50E02020190E669
:1002C600B8E06440600302035CE50F450E7003026C
:1002D600035CE490E68AF090E68BF090E6A0E020DE
:1002E600E1F990E68BE0751000F51190E6B9E0B4FF
:1002F600A335E4F512F513C3E5139511E512951030
:10030600503674402513F582E434E7F583E0FFE5C3
:100316000D2513F582E50C3512F583EFF00513E58F
:100326001370D4051280D0AD117AE779407F40ABC7
:1003360007AF0DAE0C120B91E511250DF50DE5106D
:10034600350CF50CC3E50F9511F50FE50E9510F577
:070356000E0202CFD322C307
:01035D00227D
:100CA900C0E0C083C08290E6B5E04401F0D20153B0
:0F0CB90091EF90E65D7401F0D082D083D0E032ED
:100D2F00C0E0C083C0825391EF90E65D7404F0D0B1
:060D3F0082D083D0E032F7
:100D4500C0E0C083C0825391EF90E65D7402F0D09D
:060D550082D083D0E032E1
:100AED00C0E0C083C08290E680E030E70E8521250E
:100AFD00852226852927852A28800C852925852A62
:100B0D00268521278522285391EF90E65D7410F0FC
:070B1D00D082D083D0E0324A
:100D0000C0E0C083C082D2035391EF90E65D7408C7
:080D1000F0D082D083D0E03264
:100B2400C0E0C083C08290E680E030E70E852125D6
:100B3400852226852927852A28800C852925852A2A
:100B4400268521278522285391EF90E65D7420F0B5
:070B5400D082D083D0E03213
:01003200329B
:01004200328B
:01005200327B
:010D9B003225
:010D9C003224
:010D9D003223
:010D9E003222
:010D9F003221
:010DA0003220
:010DA100321F
:010DA200321E
:010DA300321D
:010DA400321C
:010DA500321B
:010DA600321A
:010DA7003219
:010DA8003218
:010DA9003217
:010DAA003216
:010DAB003215
:010DAC003214
:010DAD003213
:010DAE003212
:010DAF003211
:010DB0003210
:010DB100320F
:010DB200320E
:010DB300320D
:010DB400320C
:010DB500320B
:010DB600320A
:010DB7003209
:010DB8003208
:010DB9003207
:010DBA003206
:010DBB003205
:040AAE00AA06AC05E3
:100AB200E4FD7E000DEE2400F582E43400F583EAC5
:100AC200F00E0D74002EF582E43400F583EFF00D84
:100AD20074002402F582E43400F583ECF07A007BA2
:0B0AE20000AF32120CE4AF32020B5BDD
:0A0B91008E148F158D168A178B182D
:100B9B00E4F519E519C3951650200515E515AE14A6
:100BAB007002051414FFE5182519F582E43517F5C5
:0A0BBB0083E0FD120AAE051980D98F
:010BC500220D
:0A0A20008E148F158D168A178B189F
:100A2A00E4FDF519E5356012E514FF7E000DEE24AC
:100A3A0000F582E43400F583EFF0AE050D74002E64
:100A4A00F582E43400F583E515F07A007B00AF32D5
:0E0A5A00120CE4AB18AA17AD16AF32020CC88E
:100C2C0090E682E030E004E020E60B90E682E030D3
:100C3C00E119E030E71590E680E04401F07F147E86
:0C0C4C0000120A6890E680E054FEF022DE
:100C840090E682E044C0F090E681F04387010000E2
:040C9400000000223A
:1000030030040990E680E0440AF0800790E680E03F
:100013004408F07FDC7E05120A6890E65D74FFF009
:0F00230090E65FF05391EF90E680E054F7F02203
:080D8700E4F51FD2E9D2AF220E
:100B5B0090E678E020E6F9C2E990E678E04480F090
:100B6B00EF25E090E679F090E678E030E0F990E65A
:100B7B0078E04440F090E678E020E6F990E678E003
:060B8B0030E1D6D2E922A0
:100BFA00A90790E678E020E6F9E51F702390E678E9
:100C0A00E04480F0E925E090E679F08D1AAF03A977
:100C1A0007751B018A1C891DE4F51E751F01D32265
:020C2A00C322E3
:100BC600A90790E678E020E6F9E51F702590E6781B
:100BD600E04480F0E925E0440190E679F08D1AAF13
:100BE60003A907751B018A1C891DE4F51E751F03E1
:040BF600D322C32221
:03004B0002058229
:10058200C0E0C083C082C085C084C086758600C0BA
:10059200D075D000C000C001C002C003C006C007B1
:1005A20090E678E030E206751F0602066C90E67867
:1005B200E020E10CE51F64026006751F0702066C6D
:1005C200E51F24FE605F14603624FE700302065DA0
:1005D20024FC70030206692408600302066CAB1B4C
:1005E200AA1CA91DAF1E051E8F8275830012068AE2
:1005F20090E679F0E51E651A7070751F05806B90A4
:10060200E679E0AB1BAA1CA91DAE1E8E8275830083
:100612001206B7751F02E51A6401704E90E678E083
:100622004420F08045E51A24FEB51E0790E678E0E6
:100632004420F0E51A14B51E0A90E678E04440F032
:10064200751F0090E679E0AB1BAA1CA91DAE1E8E99
:10065200827583001206B7051E800F90E678E0448B
:1006620040F0751F008003751F005391DFD007D043
:1006720006D003D002D001D000D0D0D086D084D012
:0806820085D082D083D0E03264
:020C5800A907EA
:100C5A00AE2DAF2E8F828E83A3E064037017AD0191
:100C6A0019ED7001228F828E83E07C002FFDEC3E0D
:090C7A00FEAF0580DF7E007F0063
:010C8300224E
:100CC800120BC6E51F24FA600E146006240770F3A1
:0C0CD800D322E4F51FD322E4F51FD32241
:100CE400120BFAE51F24FA600E146006240770F351
:0C0CF400D322E4F51FD322E4F51FD32225
:100A68008E0C8F0D90E600E054187012E50D2401ED
:100A7800FFE4350CC313F50CEF13F50D801590E664
:100A880000E05418FFBF100BE50D25E0F50DE50C4F
:100A980033F50CE50D150DAE0C7002150C4E600506
:060AA800120C9880EE2202
:100C98007400F58690FDA57C05A3E582458370F96F
:010CA8002229
:03000000020949A9
:0C094900787FE4F6D8FD75813502099036
:10068A00BB010CE58229F582E5833AF583E0225025
:10069A0006E92582F8E622BBFE06E92582F8E2226F
:0D06AA00E58229F582E5833AF583E4932289
:1006B700F8BB010DE58229F582E5833AF583E8F079
:1006C700225006E92582C8F622BBFE05E92582C825
:0206D700F2220D
:1006D900BC000BBE0029EF8DF084FFADF022E4CC05
:1006E900F875F008EF2FFFEE33FEEC33FCEE9DECCE
:1006F900984005FCEE9DFE0FD5F0E9E4CEFD22ED14
:10070900F8F5F0EE8420D21CFEADF075F008EF2F5D
:10071900FFED33FD4007985006D5F0F222C398FD4E
:050729000FD5F0EA22EB
:10072E00D083D082F8E4937012740193700DA3A35A
:10073E0093F8740193F5828883E47374029368606E
:06074E00EFA3A3A380DF6E
:100955000208B8E493A3F8E493A34003F68001F2F8
:1009650008DFF48029E493A3F85407240CC8C333A3
:10097500C4540F4420C8834004F456800146F6DF72
:10098500E4800B0102040810204080900046E47EBC
:10099500019360BCA3FF543F30E509541FFEE49367
:1009A500A360010ECF54C025E060A840B8E493A32E
:1009B500FAE493A3F8E493A3C8C582C8CAC583CA59
:1009C500F0A3C8C582C8CAC583CADFE9DEE780BE11
:01004A0000B5
:00000001FF
